:020000020000FC
:100000000BC01895FAC018951895189514C1189535
:100010001895189518951895F8940FED0DBF0FE0E9
:100020000ABBDB98D998DA98DB9800E707BBC4983D
:10003000C598C69800E10BBF80E090E000E0A02EDC
:10004000B02E789400C0C2D019D051D0FCCF07E2B6
:10005000901718F00FE0801718F4019608F0089533
:100060008FE097E2089500E0091710F4081719F0DF
:10007000019708F008958827992708959F938F93F3
:1000800006D010D020D029D08F919F91089570E094
:1000900003E0901708F408957395885E93409017D5
:1000A000D8F7089560E001E014E6901718F481177E
:1000B00008F408956395C297C29701E09017D0F7AE
:1000C0008117C0F7089550E00AE0801708F40895FA
:1000D00053958A408017E0F7089540E001E08017CB
:1000E00008F4089543958A958017E0F70895F894E9
:1000F000072F30D0112E18E011D0062F2BD0112E43
:1001000012E00CD0052F26D0112E14E007D0042FBA
:1001100021D0112E11E002D07894089507D01BBB96
:100120000000000046D011271BBB089508E0202ED8
:1001300000E0110C10F0C69801C0C69AC59A0000E4
:100140000000C5982A942016A1F7C49A0000000068
:10015000C498089510E0011711F413E00895139561
:10016000011711F41BE708951395011711F415E217
:1001700008951395011711F411E3089513950117CC
:1001800011F419E508951395011711F411E9089573
:100190001395011711F411E808951395011711F43F
:1001A0001BE308951395011711F411E0089511E16F
:1001B00008952FEF30E02A952317E9F7089503E01B
:1001C00003BF02E008BF02E009BF089502E0A016E5
:1001D00041F406B311E00123011709F402C000E065
:1001E000A02E02E0B01641F406B312E0012301177D
:1001F00009F402C000E0B02E0895F8940F931F9305
:1002000006B311E00123011739F400E0A01679F4D8
:1002100001E0A02ED4DF0BC006B312E001230117CA
:1002200031F400E0B01619F401E0B02EC8DF1F91E0
:100230000F9178941895F8940F931F9300E003BFE3
:1002400006B311E0A11651F411E00123011721F4C6
:1002500002E0A02EFCDE10C000E0A02E11E0B116DE
:1002600059F406B312E00123011721F402E0B02E85
:10027000FADE02C000E0B02E1F910F91789418951D
:00000001FF
